S01E000062696E2F64656D6F70726F675F73746D3332663330332E737265632D
S31508002000003000205D220008AB220008AD2200083F
S31508002010AF220008B1220008B32200080000000021
S31508002020000000000000000000000000B5220008C3
S31508002030B722000800000000B92200084927000856
S31508002040BD220008BF220008C1220008C3220008DA
S31508002050C5220008C7220008C9220008CB220008AA
S31508002060CD220008CF220008D1220008D32200087A
S31508002070D5220008D7220008D9220008DB2200084A
S31508002080DD220008DF220008E1220008E32200081A
S31508002090E5220008E7220008E9220008EB220008EA
S315080020A0ED220008EF220008F1220008F3220008BA
S315080020B0F5220008F722000800000000F9220008AF
S315080020C0FB2200080000000000000000FD220008B6
S315080020D000000000FF22000801230008032300086F
S315080020E00523000807230008000000000000000080
S315080020F000000000000000000000000000000000D2
S3150800210000000000000000000000000000000000C1
S315080021100000000000000000092300080B23000847
S3150800212000000000000000000000000000000000A1
S315080021300000000000000000000000000000000091
S315080021400D2300080F23000800000000000000000F
S315080021500000000000000000000000000000000071
S315080021600000000000000000000000000000000061
S315080021700000000000000000000000000000000051
S315080021800000000011230008EE11AA5510B5054CF1
S31508002190237833B9044B13B10448AFF30080012305
S315080021A0237010BD9C00002000000000703100085C
S315080021B0084B10B51BB108490848AFF3008008481A
S315080021C0036803B910BD074B002BFBD0BDE81040D0
S315080021D0184700BF00000000A0000020703100086A
S315080021E09C00002000000000154B002B08BF134B75
S315080021F09D46A3F5803A00218B460F461348144A9C
S31508002200121A00F08DFF0F4B002B00D098470E4B8B
S31508002210002B00D098470020002104000D000D482F
S31508002220002802D00C48AFF3008000F053FF2000CE
S31508002230290000F009FA00F039FF00BF0000080085
S315080022400030002000000000000000009C00002074
S315080022500C010020000000000000000007498D4620
S315080022600749084A084B9A42BEBF51F8040B42F880
S31508002270040BF8E70548804705480047003000206A
S315080022807C310008000000209C0000204530000832
S31508002290E92100081F49204A002301E041F8043BD0
S315080022A09142FBD300F0D0F9FEE7FEE7FEE7FEE732
S315080022B0FEE7FEE7FEE7FEE7FEE7FEE7FEE7FEE7E8
S315080022C0FEE7FEE7FEE7FEE7FEE7FEE7FEE7FEE7D8
S315080022D0FEE7FEE7FEE7FEE7FEE7FEE7FEE7FEE7C8
S315080022E0FEE7FEE7FEE7FEE7FEE7FEE7FEE7FEE7B8
S315080022F0FEE7FEE7FEE7FEE7FEE7FEE7FEE7FEE7A8
S31508002300FEE7FEE7FEE7FEE7FEE7FEE7FEE7FEE797
S31508002310FEE700009C0000200C010020F0B5002418
S3150800232022E0134D15F814E005EB44056F780EEB23
S31508002330070606FB00064FF4FA4595FBF6F506FB7D
S3150800234005F5B5F5FA4F0DD195FBF6F6B6B20E8042
S31508002350013EB6B2B6F5806F04D282F800E01F706F
S315080023600120F0BD0134E4B2112CDAD90020F0BD09
S315080023704831000870B588B001214FF4003000F0EC
S3150800238033FD01214FF4003000F020FD0722022121
S315080023904FF0904000F00CFE07220F214FF09040BE
S315080023A000F006FE00248DF81E4001258DF81F500A
S315080023B002268DF81C600423069303238DF81D302E
S315080023C006A94FF0904000F0A7FD8DF81C604FF469
S315080023D00043069306A94FF0904000F09DFD4FF488
S315080023E06143009301940294039405940C23049387
S315080023F0054C6946204600F013FD2946204600F0A4
S3150800240073FD08B070BD00BF0044004070B58AB0C7
S3150800241001214FF4003000F0D9FC09220B214FF0BE
S31508002420904000F0C5FD09220C214FF0904000F0C5
S31508002430BFFD4FF4C053089302238DF824300323BD
S315080024408DF8253000248DF8264001258DF8275073
S3150800245008A94FF0904000F05FFD29464FF0007044
S3150800246000F0C2FC244E304600F078F905A800F0CA
S315080024708DFA6B460DEB05020DF102014FF4FA7069
S31508002480FFF74CFF8DF81A408DF81B408DF81C405D
S315080024908DF81D408DF81E408DF81F408DF81640AA
S315080024A08DF817409DF80130013B8DF818309DF8DE
S315080024B00030013B8DF81930BDF80230ADF8143004
S315080024C005A9304600F056F98DF80E408DF80F40F4
S315080024D08DF81050ADF80440ADF80640ADF8084048
S315080024E0ADF80A40ADF80C408DF8115001A800F07F
S315080024F0D3F90AB070BD00BF0064004010B50446A9
S315080025002021064800F000FD012805D1034800F007
S31508002510F7FC2070012010BD002010BD00440040CB
S3150800252008B5FFF727FFFFF771FF08BDBFF34F8F09
S315080025300449CA6802F4E062034B1343CB60BFF355
S315080025404F8FFEE700ED00E00400FA0508B5204BC2
S315080025501B789BB91F48FFF7D1FF012836D11D4BC1
S315080025601B78002B32D000F0E9F81B4B18600122CB
S31508002570174B1A700022194B1A7008BD174B1B7897
S31508002580013314481844FFF7B9FF012814D1134A38
S3150800259013780133DBB213700E4A1278934215D1C1
S315080025A000220B4B1A700B4B5B78FF2B0ED1094B95
S315080025B09B785BB9FFF7BAFF00F0C0F8064B1B68BB
S315080025C06433984202D90022014B1A7008BD00BF35
S315080025D0FE000020BC000020B8000020FD000020FE
S315080025E000B587B00021114800F034FAD8B101AA25
S315080025F000210E4800F0DAF99DF80C3033B940F2A4
S315080026006763019A9A4203D0002302E0002300E0A0
S31508002610012343B19DF80F30FF2B04D19DF81030EC
S315080026200BB9FFF783FF07B05DF804FB00640040B1
S3150800263008B5FFF78BFFFFF7D3FF08BD08B500F015
S315080026400DF800F059F808BD08B5FFF7F7FFFFF7D2
S3150800265067FF00F025F8FFF7EBFFFAE730B583B020
S3150800266001214FF4802000F0B1FB082500950123D5
S315080026708DF8043000238DF8063003228DF80520E6
S315080026808DF80730054C6946204600F045FC29467A
S31508002690204600F08BFC03B030BD00BF00040048A4
S315080026A010B500F04BF80E4B1B68C31AB3F5FA7F4A
S315080026B014D304460B4B1B783BB90122094B1A70FD
S315080026C00821094800F070FC06E00022054B1A7044
S315080026D00821054800F06AFC014B1C6010BD00BFCC
S315080026E0000100200401002000040048014B186086
S315080026F0704700BF0801002008B50C4B1B680C4A40
S31508002700A2FB03239B09013BB3F1807F09D2094A47
S315080027105360F021084B83F82310002393600723A6
S3150800272013600020FFF7E2FF08BD00BF300000205D
S31508002730D34D621010E000E000ED00E0014B186890
S31508002740704700BF08010020024A1368013313606E
S31508002750704700BF08010020FEE700BF08B5012149
S315080027604FF0007000F04EFB00214FF0007000F0B3
S3150800277049FB08BD82B000230193036823F00203D6
S315080027800360036843F00103036002E0019B013321
S315080027900193436813F0010F04D1019A6FF07F4348
S315080027A09A42F3D1436813F0010F6FD08B79012B4E
S315080027B004D1036843F08003036003E0036823F051
S315080027C080030360CB79012B04D1036843F04003EF
S315080027D0036003E0036823F0400303600B7A012BD0
S315080027E004D1036843F02003036003E0036823F081
S315080027F0200303604B7A012B04D1036843F01003CE
S31508002800036003E0036823F0100303608B7A012B4F
S3150800281004D1036843F00803036003E0036823F068
S3150800282008030360CB7A012B04D1036843F0040341
S31508002830036003E0036823F0040303608A78CB7817
S315080028401B0643EA82730A7943EA02434A7943EA52
S3150800285002530A88013A1343C361036823F001034C
S3150800286003600023019302E0019B0133019343684F
S3150800287013F0010F04D0019A6FF07F439A42F3D107
S31508002880436813F0010F03D0002002E0002000E0A7
S31508002890012002B0704700BF70B4837A012202FAA1
S315080028A003F3394AD2F8001241F00101C2F80012C6
S315080028B0D2F81C12DC432140C2F81C12027BB2B9C2
S315080028C0314AD2F80C122140C2F80C12817AC68815
S315080028D0458845EA0645483142F83150857A868862
S315080028E0018841EA0641483502EBC5025160027B80
S315080028F0012A16D1244AD2F80C121943C2F80C122E
S31508002900817A0688458845EA0645483142F83150B5
S31508002910857A8688C18841EA0641483502EBC502B0
S315080029205160C27A32B91849D1F804222240C1F856
S31508002930042205E01449D1F804221A43C1F80422F6
S3150800294002892AB91049D1F814221440C1F8144250
S315080029500289012A05D10C49D1F814221A43C1F873
S315080029601422427B012A05D10749D1F81C221343B8
S31508002970C1F81C32044AD2F8003223F00103C2F827
S31508002980003270BC704700BF0064004000238371AA
S31508002990C371037243728372C3728370C370032355
S315080029A003710223437101230380704710B401F1B8
S315080029B01B031B01C35803F00403DBB2137233B9BC
S315080029C001F11B031B01C3585B0D136005E001F100
S315080029D01B031B01C358DB08536001F11B031B01D2
S315080029E0C418C35803F002035372636803F00F0355
S315080029F0937263681B0AD37400EB0113D3F8B841CA
S31508002A00D472D3F8B841240A1473D3F8B841240C05
S31508002A105473D3F8B841240E9473D3F8BC41D473D5
S31508002A20D3F8BC41240A1474D3F8BC41240C54745A
S31508002A30D3F8BC311B0E937421B9C36843F0200345
S31508002A40C36003E0036943F0200303615DF8044BA8
S31508002A50704700BF19B9C06800F003007047012924
S31508002A6003D1006900F0030070470020704700BFDB
S31508002A70F0B5A04B5B6803F00C03042B06D0082BBB
S31508002A8008D003BB9C4B036000241FE09A4B0360ED
S31508002A9000241BE0974B5C685A68C4F38344A31C64
S31508002AA012F4803F03D1954C04FB03F409E0914AE4
S31508002AB0D26A02F00F0201328F4CB4FBF2F404FB27
S31508002AC003F4046002E08C4B03600024894D6B68B4
S31508002AD0C3F30313DFF828E21EF80370FFB2026897
S31508002AE022FA07F343606968C1F302211EF8011050
S31508002AF0C9B223FA01F181606E68C6F3C2261EF8D0
S31508002B000660F6B2F340C360ED6A2D0905F00F0CB6
S31508002B10DFF8F0E13EF81CE01FFA8EFE15F0100F04
S31508002B2006D0BEF1000F03D0B4FBFEF5056100E048
S31508002B300261704DED6A6D0A05F00F0CDFF8C4E10D
S31508002B403EF81CE01FFA8EFE15F0100F06D0BEF1F7
S31508002B50000F03D0B4FBFEF5456100E04261654D08
S31508002B602D6B15F0100F02D1634D856100E082616F
S31508002B70604D2D6B15F0200F02D15F4DC56100E049
S31508002B80C2615C4D2D6B15F0400F02D15A4D05629E
S31508002B9000E00262574D2D6B15F4807F06D09442F3
S31508002BA004D1B74202D16500456200E04362514D47
S31508002BB02D6B15F4805F06D0944204D1B74202D13A
S31508002BC06500856200E083624A4D2D6B15F4007F2F
S31508002BD006D0944204D1B74202D16500C56200E02E
S31508002BE0C362444D2D6B15F4806F06D0944204D110
S31508002BF0B74202D16500C56400E0C3643D4D2D6B44
S31508002C0015F4006F06D0944204D1B74202D165008C
S31508002C10056500E00365374D2D6B15F4005F06D09A
S31508002C20944204D1B74202D16500456500E00365C8
S31508002C30304D2D6B15F4004F06D0944204D1B7429F
S31508002C4002D16400846500E083652A4B1B6B13F090
S31508002C50030F01D1816319E0264B1B6B03F00303B5
S31508002C60012B01D1826311E0224B1B6B03F0030396
S31508002C70022B03D14FF40043836307E01D4B1B6B04
S31508002C8003F00303032B01D11B4B8363194B1B6B07
S31508002C9013F4403F01D1C1631CE0164B1B6B03F4D0
S31508002CA04033B3F5803F01D1C26313E0114B1B6B70
S31508002CB003F44033B3F5003F03D14FF40043C36335
S31508002CC008E00C4B1B6B03F44033B3F5403F01D1CE
S31508002CD0094BC363074B1B6B13F4402F01D10164E7
S31508002CE026E0044B1B6B03F44023B3F5802F0BD16E
S31508002CF002641DE00010024000127A0000093D003F
S31508002D0020000020000000202E4B1B6B03F44023FC
S31508002D10B3F5002F03D14FF40043036408E0294BB1
S31508002D201B6B03F44023B3F5402F01D1264B0364F4
S31508002D30244B1B6B13F4401F01D141641CE0214B4B
S31508002D401B6B03F44013B3F5801F01D1426413E0F3
S31508002D501C4B1B6B03F44013B3F5001F03D14FF450
S31508002D600043436408E0174B1B6B03F44013B3F5A9
S31508002D70401F01D1144B4364124B1B6B13F4400FD5
S31508002D8001D18164F0BD0F4B1B6B03F44003B3F50F
S31508002D90800F01D18264F0BD0A4B1B6B03F440031C
S31508002DA0B3F5000F03D14FF400438364F0BD054B20
S31508002DB01B6B03F44003B3F5400F01D1024B836448
S31508002DC0F0BD00BF0010024000127A0021B1054B89
S31508002DD05A69104358617047024A536923EA00004A
S31508002DE0506170470010024021B1054BDA69104363
S31508002DF0D8617047024AD36923EA0000D061704758
S31508002E000010024021B1054B1A691043186170473A
S31508002E10024A136923EA0000106170470010024055
S31508002E2030B599B004460D46036823F001030360E4
S31508002E30436823F440528B6813434360036823F4C2
S31508002E40B05222F00C024968EB6819432B690B4310
S31508002E5013430360836823F440726B6913438360EA
S31508002E6001A8FFF705FE1C4B9C4201D10F9A0FE003
S31508002E701A4B9C4201D1109A0AE0194B9C4201D187
S31508002E80119A05E0174B9C4201D1129A00E0139A59
S31508002E90236813F4004F06D052002968B2FBF1F3F9
S31508002EA001FB132204E02968B2FBF1F301FB1322AC
S31508002EB02968B2EB510F00D30133226812F4004F90
S31508002EC006D0C3F3420223F00F031B041B0C134363
S31508002ED09BB2A38119B030BD0038014000440040C0
S31508002EE000480040004C004021B1036843F001034C
S31508002EF003607047036823F001030360704700BF4F
S31508002F00808CC0F308007047C3690B4201D00120CA
S31508002F1070470020704700BF70B400233FE00122CD
S31508002F209A400C68A24339D10A79013AD2B2012AE9
S31508002F301CD885685A000324944025EA0404846052
S31508002F4085684C7904FA02F22A4382608488A5B21D
S31508002F509AB20124944025EA040484808588ADB297
S31508002F608C7904FA02F292B22A43828004685A00E3
S31508002F70032505FA02F624EA0604046006680C79B5
S31508002F80944034430460C4689EB27600B54024EA8F
S31508002F900505CC7904FA02F22A43C26001330F2BE5
S31508002FA0BDD970BC704700BF816170470185704705
S31508002FB030B401F007039B009A40C908083150F85D
S31508002FC021400F2505FA03F324EA030340F82130CC
S31508002FD050F821301A4340F8212030BC704700BF12
S31508002FE01222164B1A60A3F580535A685A605A681B
S31508002FF05A605A6842F480625A605A6822F47C120F
S315080030005A605A6842F460125A601A6842F080722E
S315080030101A600B4B1B6813F0007FFAD0084B5A68EE
S3150800302022F003025A605A6842F002025A60044BC0
S315080030305B6803F00C03082BF9D1704700200240A7
S315080030400010024008B5154AD2F8883043F47003D8
S31508003050C2F88830124B1A6842F001021A605968A1
S31508003060104A0A405A601A6822F0847222F48032A2
S315080030701A601A6822F480221A605A6822F4FE023C
S315080030805A60DA6A22F00F02DA62196B064A0A40B7
S315080030901A6300229A60FFF7A3FF08BD00ED00E05F
S315080030A0001002400CC07FF8CCFC00FF08B5074BA7
S315080030B0044613B10021AFF30080054B1868836AF4
S315080030C003B198472046FFF747FB00BF0000000002
S315080030D06C31000870B50E4B0E4CE41AA41000258E
S315080030E01E46A54204D056F8253098470135F8E71C
S315080030F000F01EF8084C094BE41AA41000251E46D9
S31508003100A54204D056F8253098470135F8E770BD32
S3150800311094000020940000209800002094000020CD
S3150800312002440346934202D003F8011BFAE77047AC
S31508003130F8B500BFF8BC08BC9E467047F8B500BF96
S31508003140F8BC08BC9E46704705020602060307033C
S315080031500803090309040A040B040C040C050D05ED
S315080031600E050F050F06100610071008340000207C
S30908003170000000004D
S30D0800317474F0FF7F0100000062
S3150800317C010002000400060008000A000C001000FA
S3150800318C2000400080000001000000000000000044
S3150800319C00000000010203040102030406070809E3
S315080031AC0090D003000000000000000000000000A2
S315080031BC00000000000000000000000000000000F5
S315080031CC00000000000000000000000000000000E5
S315080031DC00000000000000000000000000000000D5
S315080031EC00000000000000000000000000000000C5
S315080031FC00000000000000000000000000000000B5
S3110800320C00000000B12100088D21000818
S70508002000D2
